:020000040000FA
:04000000F4EF02F027
:08000800056ED8CF06F0E0CF31
:1000100007F00001E9CF0DF0EACF08F0E1CF09F0D9
:10002000E2CF0AF0D9CF0BF0DACF0CF0F3CF14F017
:10003000F4CF15F0FACF16F000C00FF001C010F0A9
:1000400002C011F003C012F004C013F09DAA2CEFFF
:1000500000F09EBA54EF01F00FC000F010C001F0A4
:1000600011C002F012C003F013C004F00DC0E9FF8C
:1000700008C0EAFF088E09C0E1FF0AC0E2FF0BC01A
:10008000D9FF0CC0DAFF14C0F3FF15C0F4FF16C08F
:10009000FAFF055007C0E0FF06C0D8FF10003C5033
:1000A0003E02F3CF01F0F4CF00F03F02F350002600
:1000B0003D503E02F3500020026ED0EF00F03A6A4D
:1000C000386A0A0E396E376A366A3450351004E1E0
:1000D000000E016E026EE6D03A503A2A036A3424CA
:1000E000E96E35500320EA6EEFCF3BF03B502D0810
:1000F0000DE1010E386E3A503A2A036A3424E96E53
:1001000035500320EA6EEFCF3BF00DD03B502B086B
:100110000AE13A503A2A036A3424E96E3550032042
:10012000EA6EEFCF3BF03B502F08D8B0ADD03B503C
:100130003908D8A0A9D03B50300821E1036A3A50D1
:100140003424E96E35500320EA6EEF5078080AE057
:10015000036A3A503424E96E35500320EA6EEF50BA
:1001600058080DE1100E396E3A2A3A503A2A036ABD
:100170003424E96E35500320EA6EEFCF3BF039505E
:100180000A0821E13B502F081DE23B5039081AE3D1
:100190003D6A0A0E3C6E37C03FF036C03EF07FD756
:1001A000300E3B5C0124366E000E0220376E3A5052
:1001B0003A2A036A3424E96E35500320EA6EEFCF01
:1001C0003BF0E0D761D0395010085EE13B50600849
:1001D00006E23B507A0803E33B50DF0B01D03B5073
:1001E0003B6E3B502F0803E23B50390806E23B5080
:1001F00040084AE23B50460847E33B502F0819E2CB
:100200003B50390816E336343C6E37343D6E3C368D
:100210003D363C363D363C363D36F00E3C16300E13
:100220003B5C3C24016E000E3D2001C036F0376E71
:1002300016D036343C6E37343D6E3C363D363C3657
:100240003D363C363D36F00E3C16410E3B5C0A0F07
:100250003C24016E000E3D2001C036F0376E3A504E
:100260003A2A036A3424E96E35500320EA6EEF50CF
:100270003B6E600806E23B507A0803E33B50DF0B1D
:1002800001D03B503B6EADD739500A0807E1382CFE
:1002900005D0361E371E362AD8B4372A36C001F0AC
:1002A00037C002F0D7EF01F004009EAAFDD7AECF11
:1002B00032F03250DF0B336E2550080A1DE0080A79
:1002C0001BE0030A20E0020A1EE00D0A23E00E0AEA
:1002D00021E00B0A26E00D0A24E0010A29E0030AC6
:1002E0002EE00C0A33E00D0A31E00C0A36E0060A73
:1002F0003BE0030A40E047D03350530802E1252A8F
:1003000001D0256A9BD03350540802E1252A01D040
:10031000256A94D03350410802E1252A01D0256A8C
:100320008DD032503A0802E1252A01D0256A86D0C4
:100330003350510802E1252A01D0256A7FD033507D
:10034000550802E1252A01D0256A78D033504508A6
:1003500002E1252A01D0256A71D033504E0802E10E
:10036000252A01D0256A6AD03350420802E1252AA5
:1003700001D0256A63D03250200803E1252A246A7F
:1003800001D0256A5BD032500D083BE1245238E0A1
:100390002450050835E3036A24501E0FE96E000E51
:1003A0000320EA6EEF6A356A1E0E346E88D602307C
:1003B0002A6E0130296E2A3229323F0E2A16295020
:1003C0007F0B276E286A000B006E2A50010B036E0C
:1003D0000050031001E0278E000B006E2A50080B1E
:1003E000036E0050031001E02880000B006E2A50BD
:1003F000100B036E0050031001E028822680256A4E
:100400001CD0245205E13250200802E1269015D07C
:1004100032502F0811E2325039080EE324500508FB
:100420000BE3036A24501E0FE96E000E0320EA6EF0
:1004300032C0EFFF242A01D0256A00D0000E9EBAF8
:10044000010E0108D8B430D79E9A2CEF00F0700E40
:10045000D36E400E9B6ED350806A816A826A926A24
:10046000936A800E946E246A256A2690C150C00B50
:100470000F09C16EC290C66A800ED56ECD6A000E9D
:10048000CA6E000ECB6E9D8AC00EF21210EF03F002
:100490002B2AD8B42C2A2B3C0BD02C3C09D02682FA
:1004A00026748B9A26B48B8A26862C6A2B6A01D0F6
:1004B000269212EF03F0EA6A310EE96EEF5011E076
:1004C0000A0E016EBF0E006E0400002EFDD7012E35
:1004D000F9D75E0E006E002EFED700D00400EF2E7E
:1004E000EFD785EF02F08B50E30B306E2F50070BE8
:1004F000006E00360036FC0E00160050301230C080
:100500008BFF896A640E316ED6D72F500FE0010A37
:100510000FE0030A0FE0010A0FE0070A0FE0010AEB
:100520000FE0030A0FE0010A0FE010D089800FD01E
:1005300089820DD089840BD0898609D0898807D01B
:10054000898C05D0898E03D0898A01D000D0E4EF50
:1005500002F0306A8B50FC0B316E2FA001D0308A34
:100560002FA201D030882FA401D030862FA601D031
:1005700030842FA801D031802FAA01D031822FAC36
:1005800001D030802FAE01D0308231C08BFF30C01F
:100590008AFFF2EF02F0ABA202D0AB98AB8826A0A4
:1005A00021D02690285210E127500F080DE3275044
:1005B000080B006E036A0050031006E02750070B7B
:1005C0002D6E2E6A2F6E8FD7000B006E2850010BF8
:1005D000036E0050031006E027C02DF02E6A27C0DE
:1005E0002FF0B7D713EF03F0F86AD09E088EEA6AAF
:1005F000E96AB886400EAF6E030EB06EA60EAC6E02
:10060000900EAB6EC150C00B0F09C16E070EB46ED9
:10061000186A196A2692269426962B6A2C6A17D78E
:0A062000040036D7B8D7FCD703005A
:020000040030CA
:0E00000000480E0F000181000FC00FE00F40FE
:00000001FF
